:1003B60008390000000000000000082D050A0A0A9E
:0E03C6000A0A0A0A08250000000000000000D4
:10055C00E536701A75360112033C8F21E5246521AE
:0E056C00FF5521F522E521F45FF523852124BA
:01057A00225E
:10040500E535703D7535011204478F387E007C0354
:100415007DE81201D37C007D0A1201D38D2DE538CC
:1004250075F0648475F00A8485F02EE53875F00A58
:100435008475F00A8485F02FE53875F00A8485F017
:02044500302263
:01000A0022D3
:1005B200538E7F5389F0758A18758CFCC28DD28C4C
:0505C200D2A9D2AF2216
:03000B000202C22C
:1002C200C0E0C0F0C083C082C0D075D000C000C002
:1002D20001C002C003C004C005C006C0070536E560
:1002E20036640A7002F5360535AF357E00BE01066A
:1002F200BFF4037535000537E53764087002F5373A
:10030200742D2537F8E6FD74252537F8E6FBAF375F
:100312001204BD74392537F8E6FDAF37120483D0D5
:1003220007D006D005D004D003D002D001D000D02F
:0A033200D0D082D083D0F0D0E032AA
:1005C70012057B1205B212055C12040512000A809F
:0105D700F52E
:1003D4000141000142FF0143000144FF01450001C6
:0803E40046FF0147000148FF3C
:10048300ED600FA8077401088002C333D8FC424112
:10049300800EA8077401088002C333D8FCF45241CC
:1004A300E54165426013E541F4F580E5A0541F443E
:0904B30080F5A053A01F85414211
:0104BC00221D
:1004F30030000543434080035343BFE543654460F5
:1005030011854380E5A0541F44A0F5A053A01F8587
:0205130043445F
:0105150022C3
:1005160030010543451080035345EFE545654660C8
:1005260011854580E5A0541F44A0F5A053A01F8562
:02053600454638
:0105380022A0
:1005390030020543472080035347DFE5476548609C
:1005490011854780E5A0541F44A0F5A053A01F853D
:02055900474811
:01055B00227D
:1003EC000C08C0F9A4B0999282F88090FF88081488
:0803FC000102040810204080FA
:1004BD007580FFE5A0541F44E0F5A074142FF8E6F5
:1004CD00F580E5A0541F44C0F5A053A01F74082D5E
:1004DD00F8E6F580EB600353807FE5A0541F44E000
:0604ED00F5A053A01F2240
:10033C00E4FFC2A9C2C4D2C2D2B5D2B420B3027FE8
:10034C000420B2027F0520B1027F0620B0027F0795
:10035C00D2C4C2C2D2B5D2B420B3027F0820B2023A
:10036C007F0920B1027F0A20B0027F0BD2C4D2C217
:10037C00C2B5D2B420B3027F0C20B2027F0D20B1E3
:10038C00027F0E20B0027F0FD2C4D2C2D2B5C2B44B
:10039C0020B3027F1020B2027F1120B1027F122005
:0903AC00B0027F13D2A975B0FF65
:0103B5002225
:10057B007580FFE5A0541F4480F5A053A01FE4F540
:0D058B0080E5A0541F44A0F5A053A01F223E
:0600030000007F21DFFE7A
:0100090022D4
:10059800E4FEEEC3940874809480500DD29012004B
:0905A80003C2901200030E80E969
:0105B1002227
:10044700E4F5E9F5F9F5D8C2AF120598D2AFD2DED7
:1004570030910330DFFAC2DE20DF1CAFF9EFFEADCB
:10046700E9EDFFAC06E41201197B967A43798B78A4
:0B0477003C12000E020152C2DF7F00A9
:010482002257
:10000E00EC4D6011E8497017ED33EC3304600DE4EC
:10001E00FCFFFEFD22E933E8330470F80201BE1244
:10002E00018958046009E4CC248150062850090245
:10003E0001C82840030201C5C0E0EB4A7044B980F4
:10004E0006D0E0FB0201B4EF4E701CBD8008EBFF42
:10005E00EAFEE9FD80EBE98DF0A4FEE5F00200F783
:10006E00E9CDF9EAFEEBFFEF89F0A4FCE5F0CE89CD
:10007E00F0A42EFFE435F0CD89F0A42DFEE435F08A
:10008E008067EF4E7005BD80D780C3EF8BF0A4ACB8
:10009E00F0EE8BF0A42CFCE435F0F8EF8AF0A42CF3
:1000AE00E5F038FCE433CB8DF0A42CFCE5F03BF806
:1000BE00EE8AF0A42CFCE5F038F8E433CF89F0A4F6
:1000CE002CFCE5F038CF3400CE89F0A42FFFE5F0FC
:1000DE003EFEE433C98DF0A42EFEE5F039CD8AF054
:1000EE00A42FFFE5F03EFEE43DFD33D0E0FB5007CC
:1000FE000BBB000F0201C8EC2CFCEF33FFEE33FEFE
:06010E00ED33FD0201A02B
:1001140075F020800E75F010800575F0087D007E66
:10012400007F003392D530D503120228EC334010FF
:10013400EF33FFEE33FEED33FDEC33FCD5F0ED226F
:0E014400E5F0247EA2D513CC92E7CDCEFF22AB
:10015200EDD2E7CD33EC3392D524814006E4FFFEA5
:10016200FDFC22FCE4CFCECDCC24E0501174FF8004
:10017200EDC3CC13CCCD13CDCE13CECF13CF0470A1
:07018200F030D5DE02022877
:10018900E9D2E7C933E833F892D5EDD2E7CD33ECBC
:0701990033FC5002B2D52235
:1001A000EC30E7100FBF000C0EBE00080DBD0004C0
:1001B0000BEB6014A2D5EB13FCED92E7FD2274FF6C
:1001C000FCFDFEFF22E480F8A2D574FF13FC7D80C5
:0301D000E480EFD9
:03000000020236C3
:0C023600787FE4F6D8FD75814802027D57
:1001D300BC000BBE0029EF8DF084FFADF022E4CC10
:1001E300F875F008EF2FFFEE33FEEC33FCEE9DECD9
:1001F300984005FCEE9DFE0FD5F0E9E4CEFD22ED1F
:10020300F8F5F0EE8420D21CFEADF075F008EF2F68
:10021300FFED33FD4007985006D5F0F222C398FD59
:050223000FD5F0EA22F6
:0E022800C3E49FFFE49EFEE49DFDE49CFC22E7
:100242000205C7E493A3F8E493A34003F68001F206
:1002520008DFF48029E493A3F85407240CC8C333BD
:10026200C4540F4420C8834004F456800146F6DF8C
:10027200E4800B01020408102040809003B6E47E63
:10028200019360BCA3FF543F30E509541FFEE49381
:10029200A360010ECF54C025E060A840B8E493A348
:1002A200FAE493A3F8E493A3C8C582C8CAC583CA73
:1002B200F0A3C8C582C8CAC583CADFE9DEE780BE2B
:0104040000F7
:00000001FF
